:020000040000FA
:10000000012808308316023003138100831603137E
:10001000003086008312860100308B001F149F126F
:100020001F129F119F171F1383169F019F17831283
:100030000617682101308921B4200B219F1101305E
:10004000A000C62158208120CF209F150130A0009C
:10005000C621582081202A218C30A000C6211E28CC
:1000600099208030892130302E04A3213030300493
:10007000A32130302F04A32130303104A3216D306F
:10008000A3215630A32108009920C03089213030A7
:100090002E04A32130303004A32130302F04A321BB
:1000A00030303104A3216D30A3215630A321080044
:1000B0001F151F1959281E08A90083161E08831230
:1000C000A80008002608A80727080318270FA90773
:1000D0000800AD012608A802031872280130A90201
:1000E000031C2D142708A902031C2D1403102D181E
:1000F00003140800AC000310A70CA60CAC0B7B2863
:1001000008002808A6002908A700622062206220B3
:1001100062202808A6002908A70006307A20692056
:1001200001307A2069203230A6000030A700692013
:1001300008000330A700E830A600AC20AE00A701FD
:100140006430A600AC20B000A7010A30A600AC20A5
:10015000AF002808B1000800AC01AC0A6920031CFC
:10016000AD2862202C030800803089214230A32171
:100170006F30A3216F30A3217330A3217430A321EA
:100180003A30A3212030A3212030A3210D30852136
:100190004230A3216130A3217230A3210800280836
:1001A000A6002908A70001307A200030A900783085
:1001B000A80062202908AB002808AA00992008306E
:1001C00085210130AE020318FD282B08A7002A085C
:1001D000A6000330A900E830A800692099202D303E
:1001E000A32130302E04A3212C30A3213030300441
:1001F000A32130302F04A32108002B30A32130305D
:100200002E04A3212C30A32130303004A321303020
:100210002F04A3210800C03089214F30A321693069
:10022000A3216C30A3217430A3216530A3216D304C
:10023000A3217030A3213A30A3212030A321203004
:10024000A3212030A3214E308521DF30A32143306C
:10025000A321080044210130A7001130A600692025
:1002600099204B3085210130300203183A29203083
:10027000A3213D2930303004A32130302F04A321A5
:1002800030303104A32108002908AB002808AA0057
:10029000280E0F39A800290EA900F039A906A804D4
:1002A0000310A90CA80CA809A909A80A0319A90AEE
:1002B0002A08A8072B0803182B0FA9070310A90C5D
:1002C000A80C0310A90CA80C0310A90CA80C08007A
:1002D000C830A000C6213830892139308921143036
:1002E0008921553089216D308921C830A000C6216F
:1002F0007C3089210C308921013089210230A00015
:10030000C62106308921221008007F3980388921D2
:100310000800A3000830A40086100610BD21A30D1C
:1003200003188617031C86130613BD210617BD216B
:10033000A40B8F29BD218614061422180800023050
:10034000A000C6210800A3000830A40086100614EF
:10035000BD21A30D03188617031C86130613BD21A8
:100360000617BD21A40BA929BD2186140614221845
:1003700008000230A000C62108000830A5000000D7
:10038000000000000000A50BBF290800C830A10034
:10039000000000000000000000000000A10BC829C0
:0E03A000A00BC62900340000A00BD3290034A6
:02400E00223F4F
:00000001FF
